:020000040000FA
:04000000ADEF01F06F
:080008000F01ABB2AB98AB880D
:100010000E50026E0F50036E046A056A04009EBA09
:1000200013D0E86A0406055AF9E20206035A0EE301
:10003000700E046E020E056EF1D70F01ABB2AB98D5
:10004000AB8804009EAAFDD7AE50D880AAEF01F07D
:10005000E9500F0104009EA8FDD7AD6ED880AAEF2D
:1000600001F0066A076A019AA4EC01F0D8A0120018
:10007000D30FD8B4018A2D0FC60F03E20A0FF4E3A1
:1000800005D0F30FF1E2060FEFE30A0F046E040E42
:10009000056E0438E83406360736052EFBD70B4EBE
:1000A00037D0A4EC01F0D8A01200C60F03E20A0F6B
:1000B0002FE3ECD7F30F2CE2060F2AE30A0FE6D763
:1000C000066A076A019AA4EC01F0D8A01200D30FC7
:1000D000D8B4018A2D0FC60FF6E20A0FF4E3046EBE
:1000E0000A0E0602F3CF06F0F4CF02F00702F35037
:1000F0000224076E04500626D8B0072A0B4E08D0FB
:10010000A4EC01F0D8A01200C60F02E20A0FE7E249
:1001100001AA03D0E86A066C07560650D880AAEFF9
:1001200001F0019E0B50D8B4018E050E0A6E270E09
:10013000056E100E0CD8030E056EE80E08D8056A81
:10014000640E05D8056A0A0E02D8065008D0046E5F
:100150000750036E0650026E8CEC01F00250026EE6
:100160000A4E019E0B5003E00A5CD8B01200025008
:10017000D8A4019E01BE1200300FA4EF01F0080EBA
:10018000086E096E1DC0EAFF1BC0E9FF195001B4DB
:1001900020EC01F001A422EC01F01DC0E2FF1BC025
:1001A000E1FF1A50120FE96E1850EF121AC0E9FF62
:1001B000026A036A085010E001B239D8EF501814EF
:1001C000FF0F0236033601A232D8082EF5D70950A8
:1001D00001B043EF01F00250AAEF01F0080E086EE3
:1001E0001DC0EAFF1BC0E9FF195001B420EC01F06B
:1001F00001A422EC01F01DC0E2FF1BC0E1FF1A5078
:10020000120FE96E181CEF1608500FE001B043EC16
:1002100001F01AC0E9FF03320232EF501810D8A0E3
:100220001818EF6E04D8082EF6D7AAEF01F019506F
:10023000E71A000000D000D000D000D0E71A12006A
:10024000EF1203D0FF0AEF1601D0FF0AE988E92A6E
:10025000EC16AAEF01F0056A046EE86A0406055A76
:10026000D8A0AAEF01F0030E036EE60E02D8F5D770
:10027000036AFC0F026E0000E86A01D00206040067
:10028000035AFCE21200046A056A04D00332023207
:1002900004360536FF0FFAE20550036E0450026E75
:1002A000AAEF01F0D89002360336FF0FFBE20250AE
:1002B000AAEF01F0D89003320232FF0FFBE20250A6
:1002C000AAEF01F0036A056A046E010E07D0036A03
:1002D000056A046E040E02D0046E050E0A6E055007
:1002E000035C02E10450025C040ED8B0010ED8B4E5
:1002F000020E0A14D8A4FF0EAAEF01F0046E0250F9
:10030000086E0650026E0850066E0350086E0750C5
:10031000036E0850076E02D0076A066A100E086E58
:100320000334063607360450065E0550075A05E2C8
:100330000450062605500722D89002360336082EB0
:10034000EFD70250AAEF01F0E96EFB6A1350FA6E84
:100350001250F96E000104001200200EAF6E200E44
:10036000AC6E900EAB6E070EC16EF18E93909382C1
:10037000939493964B6A410E6CDE540E6ADE340EF3
:1003800068DE350E66DE200E64DE530E62DE740E0D
:1003900060DE610E5EDE720E5CDE740E5ADE690E89
:1003A00058DE6E0E56DE670E54DE2E0E52DE2E0E18
:1003B00050DE2E0E4EDE2E0E4CDE0D0E4ADE0A0EE6
:1003C00048DE246A256A406A2A6A2B6A81869396E7
:1003D000C80E41DFECEC02F0D4EF03F065EC02F064
:1003E00081969396810E1A6E0F0E1C6E010E186E7A
:1003F000810E1B6E0F0E1D6E040E196E010E016E26
:1004000040C002F0036AEADE2AC002F02BC003F00B
:10041000100EE5DE1EC002F01FC003F0DFDE040098
:1004200040506808D8B41BEF02F004004050520856
:10043000D8A433EF02F0810E1A6E0F0E1C6E010E5F
:10044000186E810E1B6E0F0E1D6E040E196E010EBE
:10045000016E026A036A100EC2DE026A036A100E9F
:10046000BEDE50EF02F0040040505608D8B43FEF13
:1004700002F0040040505408D8A450EF02F0810E5E
:100480001A6E0F0E1C6E010E186E810E1B6E0F0E73
:100490001D6E040E196E010E016E026A036A9EDE65
:1004A000120020C002F021C003F022C006F023C0D9
:1004B00007F0010E056E080E21DF2C6E03C02DF033
:1004C00006C024F007C025F01200D8902A362B363B
:1004D0001FB02A801FA02A901EC01EF01F6A1200A3
:1004E0004A6A446A81969396810E1A6E0F0E1C6EAC
:1004F000010E186E810E1B6E0F0E1D6E040E196E0E
:10050000010E016E570E026E036A68DE810E1A6ECE
:100510000F0E1C6E020E186E810E1B6E0F0E1D6EDE
:10052000040E196E020E016E2ADE496E4A060400A0
:100530004A500008D8B4A2EF02F0040049AEE6D752
:10054000E9EF02F0410E29EC00F0540E29EC00F026
:10055000340E29EC00F0350E29EC00F0440E29ECA5
:1005600000F0420E29EC00F0300E29EC00F0340EC1
:1005700029EC00F0310E29EC00F0200E29EC00F0FF
:10058000420E29EC00F0750E29EC00F0730E29ECF8
:1005900000F0790E29EC00F0200E29EC00F0450E59
:1005A00029EC00F0720E29EC00F0720E29EC00F03C
:1005B0006F0E29EC00F0720E29EC00F0210E29ECF0
:1005C00000F00D0E29EC00F00A0E29EC00F0010EEF
:1005D000446E81869396120081969396520E406ED9
:1005E0002A6A2B6A1E6A1F6AF9DE466A0400200E18
:1005F000465CD8B010EF03F0810E1A6E0F0E1C6E21
:10060000020E186E810E1B6E0F0E1D6E040E196EFB
:10061000020E016EBFEC00F03F6E462AD8A0E6D76E
:100620008186939612005CDF380E4914266E276A85
:1006300026C002F027C003F0030E3FDE266E03C083
:1006400027F0026A036A27C005F0265045DED8A4C9
:1006500074EF03F0440E29EC00F0610E29EC00F079
:10066000740E29EC00F0610E29EC00F0460E29EC26
:1006700000F06C0E29EC00F0610E29EC00F0730E16
:1006800029EC00F0680E29EC00F0200E29EC00F0B7
:10069000530E29EC00F0690E29EC00F07A0E29ECDB
:1006A00000F0650E29EC00F03D0E29EC00F0350E4F
:1006B00029EC00F0310E29EC00F0320E29EC00F0AC
:1006C0006B0E29EC00F0620E29EC00F0690E29ECAB
:1006D00000F0740E29EC00F00D0E29EC00F00A0E6B
:1006E00029EC00F0C7EF03F0010E456E2606000E60
:1006F000275A45C002F0265055EC01F0456E440ED5
:1007000029EC00F0610E29EC00F0740E29EC00F0E9
:10071000610E29EC00F0460E29EC00F06C0E29EC7D
:1007200000F0610E29EC00F0730E29EC00F0680E69
:1007300029EC00F0200E29EC00F0530E29EC00F01B
:10074000690E29EC00F07A0E29EC00F0650E29EC18
:1007500000F03D0E29EC00F00B6A45C006F0076A78
:10076000500E126E136A91EC00F06D0E29EC00F041
:10077000620E29EC00F0690E29EC00F0740E29ECF1
:1007800000F00D0E29EC00F00A0E29EC00F012002A
:100790003DC040F02CC02AF02DC02BF024C01EF02C
:1007A00025C01FF01BDE1200410E29EC00F0740E74
:1007B00029EC00F06D0E29EC00F0650E29EC00F03C
:1007C0006C0E29EC00F0200E29EC00F0410E29EC13
:1007D00000F0540E29EC00F0340E29EC00F0350E38
:1007E00029EC00F0440E29EC00F0420E29EC00F058
:1007F000300E29EC00F0340E29EC00F0310E29EC1B
:1008000000F0200E29EC00F0440E29EC00F0650EFB
:1008100029EC00F06D0E29EC00F06F0E29EC00F0D1
:100820000D0E29EC00F00A0E29EC00F03D0E29EC2B
:1008300000F03D0E29EC00F03D0E29EC00F03D0EDD
:1008400029EC00F03D0E29EC00F03D0E29EC00F003
:100850003D0E29EC00F03D0E29EC00F03D0E29EC98
:1008600000F03D0E29EC00F03D0E29EC00F03D0EAD
:1008700029EC00F03D0E29EC00F03D0E29EC00F0D3
:100880003D0E29EC00F03D0E29EC00F03D0E29EC68
:1008900000F03D0E29EC00F03D0E29EC00F03D0E7D
:1008A00029EC00F00D0E29EC00F00A0E29EC00F006
:1008B000BADE0D0E29EC00F00A0E29EC00F0410E14
:1008C00029EC00F0740E29EC00F06D0E29EC00F01C
:1008D000650E29EC00F06C0E29EC00F0200E29ECDE
:1008E00000F0440E29EC00F0610E29EC00F0740ECB
:1008F00029EC00F0610E29EC00F0460E29EC00F026
:100900006C0E29EC00F0610E29EC00F0730E29EC5E
:1009100000F0680E29EC00F0200E29EC00F0440EE7
:1009200029EC00F0650E29EC00F06D0E29EC00F0CA
:100930006F0E29EC00F00D0E29EC00F00A0E29ECE8
:1009400000F0570E29EC00F0610E29EC00F0690E62
:1009500029EC00F0740E29EC00F0690E29EC00F08F
:100960006E0E29EC00F0670E29EC00F0200E29EC49
:1009700000F0660E29EC00F06F0E29EC00F0720E0C
:1009800029EC00F0200E29EC00F0640E29EC00F0B8
:10099000610E29EC00F0740E29EC00F0610E29ECD8
:1009A00000F02E0E29EC00F02E0E29EC00F02E0E99
:1009B00029EC00F02E0E29EC00F00D0E29EC00F0D1
:1009C0000A0E29EC00F04F0E29EC00F0700E29EC15
:1009D00000F0740E29EC00F0690E29EC00F06F0EA7
:1009E00029EC00F06E0E29EC00F0730E29EC00F0FB
:1009F0003A0E29EC00F00D0E29EC00F00A0E29EC5D
:100A000000F0310E29EC00F0200E29EC00F02D0E44
:100A100029EC00F0200E29EC00F0520E29EC00F039
:100A2000650E29EC00F0610E29EC00F0640E29EC53
:100A300000F0200E29EC00F0660E29EC00F0720E9A
:100A400029EC00F06F0E29EC00F06D0E29EC00F09F
:100A5000200E29EC00F0610E29EC00F0640E29EC68
:100A600000F0640E29EC00F0720E29EC00F0650E27
:100A700029EC00F0730E29EC00F0730E29EC00F065
:100A80000D0E29EC00F00A0E29EC00F0320E29ECD4
:100A900000F0200E29EC00F02D0E29EC00F0200EC5
:100AA00029EC00F0570E29EC00F0720E29EC00F052
:100AB000690E29EC00F0740E29EC00F0650E29ECAB
:100AC00000F0200E29EC00F0740E29EC00F06F0EFF
:100AD00029EC00F0200E29EC00F0610E29EC00F06A
:100AE000640E29EC00F0640E29EC00F0720E29EC83
:100AF00000F0650E29EC00F0730E29EC00F0730E87
:100B000029EC00F0200E29EC00F0650E29EC00F035
:100B1000720E29EC00F0610E29EC00F0730E29EC46
:100B200000F0650E29EC00F0200E29EC00F0660EB6
:100B300029EC00F0690E29EC00F0720E29EC00F0AF
:100B4000730E29EC00F0740E29EC00F00D0E29EC68
:100B500000F00A0E29EC00F0330E29EC00F0200E14
:100B600029EC00F02D0E29EC00F0200E29EC00F00D
:100B7000570E29EC00F0720E29EC00F0690E29ECFA
:100B800000F0740E29EC00F0650E29EC00F0200E48
:100B900029EC00F0740E29EC00F06F0E29EC00F047
:100BA000200E29EC00F0610E29EC00F0640E29EC17
:100BB00000F0640E29EC00F0720E29EC00F0650ED6
:100BC00029EC00F0730E29EC00F0730E29EC00F014
:100BD000200E29EC00F06E0E29EC00F06F0E29ECCF
:100BE00000F0200E29EC00F0650E29EC00F0720EEA
:100BF00029EC00F0610E29EC00F0730E29EC00F0F6
:100C0000650E29EC00F00D0E29EC00F00A0E29EC1F
:100C100000F0340E29EC00F0200E29EC00F02D0E2F
:100C200029EC00F0200E29EC00F0570E29EC00F022
:100C3000720E29EC00F0690E29EC00F0740E29EC1C
:100C400000F0650E29EC00F02F0E29EC00F0520E9A
:100C500029EC00F0650E29EC00F0610E29EC00F0A3
:100C6000640E29EC00F0200E29EC00F0540E29EC63
:100C700000F0650E29EC00F0730E29EC00F0740E04
:100C800029EC00F0200E29EC00F0610E29EC00F0B8
:100C9000740E29EC00F0200E29EC00F0610E29EC16
:100CA00000F0640E29EC00F0640E29EC00F0720EE6
:100CB00029EC00F0650E29EC00F0730E29EC00F031
:100CC000730E29EC00F00D0E29EC00F00A0E29EC51
:100CD00000F00D0E29EC00F00A0E29EC00F0410E98
:100CE00029EC00F0640E29EC00F0640E29EC00F011
:100CF000720E29EC00F0650E29EC00F0730E29EC61
:100D000000F0730E29EC00F0200E29EC00F06D0EBF
:100D100029EC00F0750E29EC00F0730E29EC00F0C0
:100D2000740E29EC00F0200E29EC00F0620E29EC84
:100D300000F0650E29EC00F0200E29EC00F0610EA9
:100D400029EC00F0200E29EC00F0640E29EC00F0F4
:100D50006F0E29EC00F0750E29EC00F0620E29EC04
:100D600000F06C0E29EC00F0650E29EC00F0200E6E
:100D700029EC00F0770E29EC00F06F0E29EC00F062
:100D8000720E29EC00F0640E29EC00F0200E29EC24
:100D900000F0690E29EC00F06E0E29EC00F0200E38
:100DA00029EC00F0680E29EC00F0650E29EC00F04B
:100DB000780E29EC00F00D0E29EC00F00A0E29EC5B
:100DC00000F0540E29EC00F0680E29EC00F0650EDE
:100DD00029EC00F0200E29EC00F07E0E29EC00F04A
:100DE000200E29EC00F0280E29EC00F0740E29ECFE
:100DF00000F0690E29EC00F06C0E29EC00F0640E96
:100E000029EC00F0650E29EC00F0290E29EC00F029
:100E1000200E29EC00F0690E29EC00F0730E29EC8D
:100E200000F0200E29EC00F0750E29EC00F0730E96
:100E300029EC00F0650E29EC00F0640E29EC00F0BE
:100E4000200E29EC00F0610E29EC00F0730E29EC65
:100E500000F0200E29EC00F0610E29EC00F0200ECD
:100E600029EC00F0730E29EC00F0740E29EC00F070
:100E7000610E29EC00F0720E29EC00F0740E29ECE2
:100E800000F02F0E29EC00F0730E29EC00F0740E28
:100E900029EC00F06F0E29EC00F0700E29EC00F048
:100EA000200E29EC00F0630E29EC00F06F0E29EC07
:100EB00000F0640E29EC00F0650E29EC00F00D0E38
:100EC00029EC00F00A0E29EC00F0660E29EC00F087
:100ED0006F0E29EC00F06C0E29EC00F06C0E29EC82
:100EE00000F06F0E29EC00F0770E29EC00F0650E93
:100EF00029EC00F0640E29EC00F0200E29EC00F043
:100F0000620E29EC00F0790E29EC00F0200E29EC9D
:100F100000F0740E29EC00F0680E29EC00F0650E6C
:100F200029EC00F0200E29EC00F06F0E29EC00F007
:100F3000700E29EC00F0740E29EC00F0690E29EC1B
:100F400000F06F0E29EC00F06E0E29EC00F0200E80
:100F500029EC00F0610E29EC00F06E0E29EC00F097
:100F6000640E29EC00F0200E29EC00F0740E29EC40
:100F700000F0680E29EC00F0650E29EC00F0200E60
:100F800029EC00F0610E29EC00F0640E29EC00F071
:100F9000640E29EC00F0720E29EC00F0650E29ECCD
:100FA00000F0730E29EC00F0730E29EC00F00D0E2A
:100FB00029EC00F00A0E29EC00F0450E29EC00F0B7
:100FC000780E29EC00F0610E29EC00F06D0E29EC92
:100FD00000F0700E29EC00F06C0E29EC00F0650EAC
:100FE00029EC00F03A0E29EC00F0200E29EC00F07C
:100FF0007E0E29EC00F0310E29EC00F0300E29ECC9
:1010000000F0300E29EC00F0300E29EC00F0340E28
:1010100029EC00F0320E29EC00F0300E29EC00F043
:10102000300E29EC00F0300E29EC00F00D0E29EC0A
:1010300000F00A0E29EC00F0770E29EC00F0690EA2
:1010400029EC00F06C0E29EC00F06C0E29EC00F09D
:10105000200E29EC00F0720E29EC00F0650E29EC50
:1010600000F0610E29EC00F0640E29EC00F0200E77
:1010700029EC00F0640E29EC00F0610E29EC00F080
:10108000740E29EC00F0610E29EC00F0200E29EC22
:1010900000F0620E29EC00F0650E29EC00F0670EFE
:1010A00029EC00F0690E29EC00F06E0E29EC00F03E
:1010B0006E0E29EC00F0690E29EC00F06E0E29ECA2
:1010C00000F0670E29EC00F0200E29EC00F0610E14
:1010D00029EC00F0740E29EC00F0200E29EC00F051
:1010E000680E29EC00F0650E29EC00F0780E29EC72
:1010F00000F0200E29EC00F0300E29EC00F0300E4C
:1011000029EC00F0300E29EC00F0340E29EC00F050
:10111000320E29EC00F0300E29EC00F0300E29ECF4
:1011200000F0300E29EC00F00D0E29EC00F00A0E54
:1011300029EC00F01DEC00F07E08D8A4FBD7010ECE
:101140000B6E3A0E126E136A60EC00F0476E040EDE
:101150000B6E3A0E126E136A31EC00F0206E07C06F
:1011600021F0040E0B6E3A0E126E136A31EC00F091
:10117000226E07C023F051EC02F00A0E29EC00F0B9
:101180000D0E29EC00F0500E29EC00F0610E29EC58
:1011900000F0670E29EC00F0650E29EC00F03A0E25
:1011A00029EC00F00B6A2CC006F02DC007F0500EA1
:1011B000126E136A91EC00F0200E29EC00F0410E43
:1011C00029EC00F0640E29EC00F0640E29EC00F02C
:1011D000720E29EC00F03A0E29EC00F00B6A24C0E4
:1011E00006F025C007F0500E126E136A91EC00F065
:1011F0000D0E29EC00F00A0E29EC00F00400475017
:101200000108D8B445EF09F0040047500208D8B4EB
:10121000F1EF09F0040047500308D8B4F1EF09F0EA
:10122000040047500408D8B4A3EF0AF04F0E29EC8D
:1012300000F0700E29EC00F0740E29EC00F0690E3D
:1012400029EC00F06F0E29EC00F06E0E29EC00F096
:10125000200E29EC00F0450E29EC00F0720E29EC6E
:1012600000F0720E29EC00F06F0E29EC00F0720E07
:1012700029EC00F0210E29EC00F00D0E29EC00F015
:101280000A0E29EC00F059EF04F0520E406E2CC00B
:101290002AF02DC02BF024C01EF025C01FF0EEEC6C
:1012A00001F00D0E29EC00F00A0E29EC00F0500EB2
:1012B00029EC00F0610E29EC00F0670E29EC00F03B
:1012C000650E29EC00F03A0E29EC00F00B6A2CC0F8
:1012D00006F02DC007F0500E126E136A91EC00F06C
:1012E0000D0E29EC00F00A0E29EC00F0010E466EFE
:1012F000810E1A6E0F0E1C6E020E186E810E1B6E82
:101300000F0E1D6E040E196E020E016EBFEC00F082
:101310003F6E0400800E3F5CD8A091EF09F02E0EC6
:101320003F6E0400200E3F5CD8B099EF09F02E0EFE
:101330003F6E3F5029EC00F0462AD8A0D9D78186CD
:1013400093960D0E29EC00F00A0E29EC00F04D0EDC
:1013500029EC00F06F0E29EC00F0720E29EC00F081
:10136000650E29EC00F03F0E29EC00F0200E29EC70
:1013700000F0310E29EC00F03D0E29EC00F0790E62
:1013800029EC00F0650E29EC00F0730E29EC00F05A
:10139000200E29EC00F0320E29EC00F03D0E29EC75
:1013A00000F06E0E29EC00F06F0E29EC00F00D0E2F
:1013B00029EC00F00A0E29EC00F0010E0B6E3A0E3B
:1013C000126E136A60EC00F03F6E04003F5001089B
:1013D000D8A459EF04F02C2A000E2D2256D759EF2D
:1013E00004F0450E29EC00F06E0E29EC00F0740EAE
:1013F00029EC00F0650E29EC00F0720E29EC00F0EB
:10140000200E29EC00F0740E29EC00F0650E29EC9A
:1014100000F0780E29EC00F0740E29EC00F0200E9C
:1014200029EC00F07E0E29EC00F0200E29EC00F0F3
:10143000280E29EC00F0740E29EC00F0690E29EC5E
:1014400000F06C0E29EC00F0640E29EC00F0650E43
:1014500029EC00F0290E29EC00F0200E29EC00F018
:10146000740E29EC00F06F0E29EC00F0200E29EC30
:1014700000F0650E29EC00F06E0E29EC00F0640E11
:1014800029EC00F00D0E29EC00F00A0E29EC00F01A
:10149000840E406E24C01EF025C01FF0EEEC01F05B
:1014A000E80E0E6E030E0F6E04EC00F0D8A0F8D715
:1014B0003F6E3FC002F0200E67EC01F0146E3FC09B
:1014C00002F07F0E62EC01F0166E14501610D8A4D4
:1014D000E7D704003F507E08D8B483EF0AF0810EAE
:1014E0001A6E0F0E1C6E010E186E810E1B6E0F0E03
:1014F0001D6E040E196E010E016E3FC002F0036AEC
:10150000EEEC00F0CDD78186939604004750020898
:10151000D8A48DEF0AF0830E406E040047500308F4
:10152000D8A495EF0AF0880E406E2CC02AF02DC08A
:101530002BF0EEEC01F08186939670EC02F0818640
:10154000939659EF04F0570E29EC00F0720E29EC37
:1015500000F0690E29EC00F0740E29EC00F0690E21
:1015600029EC00F06E0E29EC00F0670E29EC00F07B
:10157000200E29EC00F0730E29EC00F0610E29EC2E
:1015800000F06D0E29EC00F0700E29EC00F06C0EEE
:1015900029EC00F0650E29EC00F0200E29EC00F09B
:1015A000740E29EC00F0650E29EC00F0780E29ECA1
:1015B00000F0740E29EC00F0200E29EC00F0740EFF
:1015C00029EC00F06F0E29EC00F0200E29EC00F061
:1015D000420E29EC00F0750E29EC00F0660E29ECA5
:1015E00000F0660E29EC00F0650E29EC00F0720E9A
:1015F00029EC00F0200E29EC00F0310E29EC00F06F
:101600003A0E29EC00F00B6A2CC006F02DC007F052
:10161000500E126E136A91EC00F0200E29EC00F0CF
:10162000610E29EC00F0740E29EC00F0200E29EC7C
:1016300000F0410E29EC00F0640E29EC00F0640E7D
:1016400029EC00F0720E29EC00F0650E29EC00F098
:10165000730E29EC00F0730E29EC00F03A0E29EC21
:1016600000F00B6A24C006F025C007F0500E126E81
:10167000136A91EC00F00D0E29EC00F00A0E29EC33
:1016800000F0840E406E24C01EF025C01FF0EEEC6A
:1016900001F03E0E286E296A466A46C002F0036ACF
:1016A00029C005F0285064EC01F0D8A4C7EF0BF076
:1016B0004650F66E3F08D8A0AEEF0BF0F76AF86A16
:1016C000D890F636F736DC0EF626160EF722000E08
:1016D000F8220800F5CF3FF0AEEF0BF0570C650C89
:1016E0006C0C630C6F0C6D0C650C210C200C540CF5
:1016F000680C690C730C200C690C730C200C610CC9
:101700006E0C200C410C740C6D0C650C6C0C200CD8
:10171000410C540C340C350C440C420C300C340C81
:10172000310C420C200C340C6D0C620C690C740CE6
:10173000200C640C610C740C610C660C6C0C610C5C
:10174000730C680C200C380C200C700C690C6E0C9F
:10175000200C630C680C690C700C210C810E1A6E45
:101760000F0E1C6E010E186E810E1B6E0F0E1D6E7D
:10177000040E196E010E016E3FC002F0036AEEEC1A
:1017800000F03F5029EC00F0462AD8A086D7818689
:1017900093960D0E29EC00F00A0E29EC00F0520E83
:1017A00029EC00F0650E29EC00F0610E29EC00F048
:1017B000640E29EC00F0690E29EC00F06E0E29ECA5
:1017C00000F0670E29EC00F0200E29EC00F0620E0C
:1017D00029EC00F0610E29EC00F0630E29EC00F01A
:1017E0006B0E29EC00F0200E29EC00F0620E29ECC3
:1017F00000F0750E29EC00F0660E29EC00F0660E84
:1018000029EC00F0650E29EC00F0720E29EC00F0D6
:101810002E0E29EC00F02E0E29EC00F02E0E29ECF5
:1018200000F00D0E29EC00F00A0E29EC00F0540E29
:10183000406E24C01EF025C01FF0EEEC01F0466A99
:1018400046C002F0036A29C005F0285064EC01F09C
:10185000D8A442EF0CF0810E1A6E0F0E1C6E020E11
:10186000186E810E1B6E0F0E1D6E040E196E020E89
:10187000016EBFEC00F03F6E3F5029EC00F0462AAD
:10188000D8A0DED7818693960D0E29EC00F00A0EC3
:1018900029EC00F0450E29EC00F0720E29EC00F066
:1018A000610E29EC00F0730E29EC00F0650E29ECB6
:1018B00000F0200E29EC00F0260E29EC00F0200E9E
:1018C00029EC00F0770E29EC00F0720E29EC00F004
:1018D000690E29EC00F0740E29EC00F0650E29EC7D
:1018E00000F0200E29EC00F0740E29EC00F06F0ED1
:1018F00029EC00F0200E29EC00F0440E29EC00F059
:10190000610E29EC00F0740E29EC00F0610E29EC58
:1019100000F0460E29EC00F06C0E29EC00F0610E90
:1019200029EC00F0730E29EC00F0680E29EC00F0B1
:10193000200E29EC00F0730E29EC00F0650E29EC66
:1019400000F0630E29EC00F0740E29EC00F06F0E2D
:1019500029EC00F0720E29EC00F02E0E29EC00F0BC
:101960002E0E29EC00F02E0E29EC00F00D0E29ECC5
:1019700000F00A0E29EC00F0830E406E2CC02AF015
:101980002DC02BF0EEEC01F08186939670EC02F006
:1019900081869396520E29EC00F0650E29EC00F03A
:1019A000610E29EC00F0640E29EC00F0690E29ECC0
:1019B00000F06E0E29EC00F0670E29EC00F0200E0E
:1019C00029EC00F0620E29EC00F0610E29EC00F029
:1019D000630E29EC00F06B0E29EC00F0200E29ECD0
:1019E00000F0440E29EC00F0610E29EC00F0740EBA
:1019F00029EC00F0610E29EC00F0460E29EC00F015
:101A00006C0E29EC00F0610E29EC00F0730E29EC4D
:101A100000F0680E29EC00F0200E29EC00F0730EA7
:101A200029EC00F0650E29EC00F0630E29EC00F0C3
:101A3000740E29EC00F06F0E29EC00F0720E29EC08
:101A400000F02E0E29EC00F02E0E29EC00F02E0EE8
:101A500029EC00F00D0E29EC00F00A0E29EC00F044
:101A6000520E406E2CC02AF02DC02BF024C01EF068
:101A700025C01FF0EEEC01F0466A46C002F0036A92
:101A800029C005F0285064EC01F0D8A45FEF0DF0F8
:101A9000810E1A6E0F0E1C6E020E186E810E1B6EDA
:101AA0000F0E1D6E040E196E020E016EBFEC00F0DB
:101AB0003F6E3F5029EC00F0462AD8A0DED7818641
:101AC00093960D0E29EC00F00A0E29EC00F0460E5C
:101AD00029EC00F0690E29EC00F06E0E29EC00F004
:101AE000690E29EC00F0730E29EC00F0680E29EC69
:101AF00000F0650E29EC00F0640E29EC00F00D0EEC
:101B000029EC00F00A0E29EC00F059EF04F0040073
:061B1000FED70300FED722
:020000040030CA
:08000000FF321FF3FFF98BFF33
:00000001FF
